:020000040800F2
:10000000002000207901000889010008890100080A
:1000100000000000000000000000000000000000E0
:10002000000000000000000000000000890100083E
:10003000000000000000000089010008890100089C
:100040008901000889010008890100088901000868
:100050008901000889010008890100088901000858
:100060008901000889010008890100088901000848
:100070008901000889010008890100088901000838
:1000800089010008890100080000000089010008BA
:100090008901000889010008890100088901000818
:1000A0008901000889010008890100088901000808
:1000B000890100080000000089010008000000001C
:0400C0005FF808F1EC
:1000C40080B500AF074B074A5269802109030A43F0
:1000D4005A61054B044A1268A02149030A431A6075
:1000E400BD4680BD001002400008004880B584B0C1
:1000F40000AF78607B68FB60C046FB681A1C511E29
:100104008A41D2B2013BFB60002AF6D1BD4604B05D
:1001140080BDC04680B500AF024B802292009A6138
:10012400BD4680BD0008004880B500AF024B802268
:1001340092049A61BD4680BD0008004880B500AFB6
:10014400FFF7E8FF054B181CFFF7D0FFFFF7ECFFA4
:10015400024B181CFFF7CAFFF2E7C046400D03002C
:100164008C01000800000020000000200000002096
:1001740000000020C046C046C046FFF7A1FFFFF7BD
:08018400DDFF7047FEE70000FB
:040000050800017975
:00000001FF
